:040000008A11112828
:10000800FE00030E83120313CB000408CC000A0879
:10001800CD007F08CE008A15902C8A115C28A1306B
:100028009F0083169F133C208A111F151F191A2839
:100038001E08080099309F0083169F133C208A11E0
:100048001F151F1925281E08080091309F008316C8
:100058009F173C208A111F151F1930281E08D10030
:10006800D00183161E088312D0070318D10A08008E
:100078008312CF013230CF0A4F02031808003E28FE
:100088008A15FE2C8A15342D8A155B2D8A15722D3A
:100098008A157D2D8A159D2D8A15BE2D8A15E22D6E
:1000A8008A15132E8A15362E8A15392E8A15472E4B
:1000B8002030FD01E2018313840042308A11A3201D
:1000C8008A11AE308400B5308A11A32083018A15C5
:1000D8005B2AD100D0014F085118D0070310CF0D6B
:1000E8000310D10CD108031D6F28500808004930AF
:1000F8008B12831290009010901183160C148312A7
:10010800101408001C3083169B001F1783128030C0
:100118001F1783169F0008007C3083168F003C3021
:1001280085003B3086008330810008008B170B1751
:100138008B118C120C1201130B168B120800640021
:0E0148008001840A0406031900340406A4286A
:10020000FF1B0A2983137F1883170008840A031928
:10021000FF0A08007F087F398A000408840A03194E
:10022000FF0A82000034003413340134E534013411
:10023000903402341F3403349B34033408340434C0
:100240006A340434C2340434123405345B34053463
:100250009F340534DF3405341A34063452340634FE
:1002600086340634B7340634E6340634133407349F
:100270003E340734663407348D340734B2340734DF
:10028000D6340734F93407341A3408343A3408348D
:10029000593408347734083494340834B03408348A
:1002A000CB340834E5340834FF34083418340934C6
:1002B00030340934483409345F340934763409342D
:1002C0008C340934A1340934B6340934CA340934BD
:1002D000DE340934F234093405340A3418340A346B
:1002E0002A340A343C340A344E340A345F340A3433
:1002F00070340A3481340A3491340A34A2340A3412
:10030000B1340A34C1340A34D0340A34DF340A3404
:10031000EE340A34FD340A340B340B3419340B3404
:1003200027340B3435340B3442340B344F340B3414
:100330005C340B3469340B3476340B3483340B3433
:100340008F340B349B340B34A7340B34B3340B345D
:10035000BF340B34CA340B34D6340B34E1340B3491
:10036000EC340B34F7340B3402340C340D340C34CD
:1003700018340C3422340C342C340C3437340C3410
:1003800041340C344B340C3455340C345F340C345D
:1003900068340C3472340C347C340C3485340C34B2
:1003A0008E340C3498340C34A1340C34AA340C340C
:1003B000B3340C34BC340C34C4340C34CD340C346D
:1003C000D6340C34DE340C34E7340C34EF340C34D3
:1003D000F7340C3400340D3408340D3410340D343B
:1003E00018340D3420340D3428340D342F340D34AA
:1003F00037340D343F340D3446340D344E340D341F
:1004000055340D345D340D3464340D346B340D3497
:1004100073340D347A340D3481340D3488340D3412
:100420008F340D3496340D349D340D34A4340D3492
:10043000AB340D34B1340D34B8340D34BF340D3415
:10044000C5340D34CC340D34D2340D34D9340D349C
:10045000DF340D34E6340D34EC340D34F2340D3425
:10046000F8340D34FF340D3405340E340B340E34AF
:1004700011340E3417340E341D340E3423340E343C
:1004800029340E342F340E3435340E343A340E34CD
:1004900040340E3446340E344C340E3451340E3461
:1004A00057340E345D340E3462340E3468340E34F6
:1004B0006D340E3473340E3478340E347D340E348F
:1004C00083340E3488340E348D340E3493340E3429
:1004D00098340E349D340E34A2340E34A7340E34C6
:1004E000AC340E34B2340E34B7340E34BC340E3463
:1004F000C1340E34C6340E34CB340E34D0340E3402
:10050000D4340E34D9340E34DE340E34E3340E34A5
:10051000E8340E34EC340E34F1340E34F6340E3448
:10052000FB340E34FF340E3404340F3409340F34EA
:100530000D340F3412340F3416340F341B340F348F
:100540001F340F3424340F3428340F342D340F3437
:1005500031340F3436340F343A340F343E340F34E0
:1005600043340F3447340F344B340F344F340F348B
:1005700054340F3458340F345C340F3460340F3437
:1005800065340F3469340F346D340F3471340F34E3
:1005900075340F3479340F347D340F3481340F3493
:1005A00085340F3489340F348D340F3491340F3443
:1005B00095340F3499340F349D340F34A1340F34F3
:1005C000A5340F34A9340F34AD340F34B0340F34A4
:1005D000B4340F34B8340F34BC340F34C0340F3457
:1005E000C3340F34C7340F34CB340F34CF340F340B
:1005F000D2340F34D6340F34DA340F34DD340F34C0
:10060000E1340F34E5340F34E8340F34EC340F3474
:10061000EF340F34F3340F34F6340F34FA340F342C
:10062000FD340F340034003400340034013400341D
:10063000013400340234003404340034063400340D
:10064000083400340A3400340D34003410340034DB
:1006500013340034163400341A3400341E34003499
:1006600023340034283400342D3400343234003440
:10067000383400343E340034443400344B340034D5
:100680005234003459340034603400346834003457
:100690007034003479340034813400348A340034C6
:1006A000933400349D340034A7340034B134003422
:1006B000BB340034C6340034D1340034DC3400346C
:1006C000E8340034F4340034003401340C340134A0
:1006D00019340134253401343334013440340134C5
:1006E0004E3401345C3401346A34013478340134DA
:1006F0008734013496340134A5340134B5340134DF
:10070000C4340134D4340134E4340134F5340134D4
:1007100005340234163402342734023439340234B6
:100720004A3402345C3402346E340234803402348D
:1007300093340234A5340234B8340234CB34023456
:10074000DE340234F2340234063403341934033410
:100750002D34033442340334563403346B340334BD
:100760007F34033494340334A9340334BF34033462
:10077000D4340334EA3403340034043415340434F8
:100780002B34043442340434583404346F34043485
:10079000853404349C340434B3340434CA3404340B
:1007A000E1340434F8340434103405342734053487
:1007B0003F340534573405346F34053486340534FA
:1007C0009E340534B7340534CF340534E73405346A
:1007D000FF340534183406343034063449340634D2
:1007E000623406347A34063493340634AC34063436
:1007F000C5340634DE340634F73406341034073496
:1008000029340734423407345B34073474340734F2
:100810008E340734A7340734C0340734D93407344E
:10082000F23407340C340834253408343E340834A8
:1008300057340834703408348A340834A334083404
:10084000BC340834D5340834EE3408340734093461
:100850002034093439340934523409346B340934BE
:10086000843409349C340934B5340934CE34093421
:10087000E6340934FF34093417340A342F340A3487
:1008800047340A3460340A3478340A348F340A34F2
:10089000A7340A34BF340A34D7340A34EE340A3465
:1008A00006340B341D340B3434340B344B340B34DA
:1008B00062340B3479340B348F340B34A6340B345C
:1008C000BC340B34D3340B34E9340B34FF340B34E5
:1008D00014340C342A340C343F340C3455340C3476
:1008E0006A340C347F340C3493340C34A8340C3414
:1008F000BC340C34D1340C34E5340C34F8340C34BE
:100900000C340D3420340D3433340D3446340D346E
:1009100059340D346B340D347E340D3490340D3431
:10092000A2340D34B4340D34C5340D34D7340D3401
:10093000E8340D34F9340D3409340E341A340E34DD
:100940002A340E343A340E3449340E3459340E34C9
:1009500068340E3477340E3486340E3494340E34C6
:10096000A2340E34B0340E34BE340E34CB340E34D4
:10097000D9340E34E5340E34F2340E34FE340E34F1
:100980000A340F3416340F3422340F342D340F341C
:1009900038340F3443340F344D340F3457340F345C
:1009A00061340F346B340F3474340F347D340F34AE
:1009B00085340F348E340F3496340F349E340F3414
:1009C000A5340F34AC340F34B3340F34BA340F348D
:1009D000C0340F34C6340F34CC340F34D1340F3418
:1009E000D6340F34DB340F34E0340F34E4340F34B6
:1009F000E8340F34EB340F34EE340F34F1340F3469
:100A0000F4340F34F6340F34F8340F34FA340F342E
:100A1000FC340F34FD340F34FD340F34FE340F3406
:100A2000FE340F3404340434043404340434043401
:100A300004340434043404340434043405340534F4
:100A400005340534053405340534053405340534DE
:100A500005340534053405340534053405340534CE
:100A600005340534053405340534053405340534BE
:100A700005340534053405340534053405340534AE
:100A8000053405340534053405340634063406349B
:100A90000634063406340634063406340634063486
:100AA0000634063406340634063406340634063476
:100AB0000634063406340634063406340634063466
:100AC0000634063406340634063407340734073453
:100AD000073407340734073407340734073407343E
:100AE000073407340734073407340734073407342E
:100AF000073407340734073407340734073407341E
:100B00000734083408340834083408340834083406
:100B100008340834083408340834083408340834F5
:100B200008340834083408340834083408340834E5
:100B300008340834093409340934093409340934CF
:100B40000934093409340934B934BF34C534CB34D9
:100B5000D034D634DC34E234E834EE34F434FA34CD
:100B6000013407340D3413341934203426342C3432
:100B7000323439343F3445344C34523459345F3490
:100B800066346C3473347934803487348D349434DF
:100B90009B34A234A934AF34B634BD34C434CB341E
:100BA000D234D934E034E834EF34F634FD3406344A
:100BB0000D3414341C3423342A343234393441345F
:100BC000493450345834603467346F3477347F3468
:100BD00087348F3497349F34A734AF34B734BF345D
:100BE000C734CF34D834E034E834F134F934033442
:100BF0000B3414341C3425342D3436343F3448340B
:100C00005134593462346B3474347D3487349034C5
:100C10009934A234AB34B534BE34C734D134DA3469
:100C2000E434ED34F73402340B3415341F342934F2
:100C300033343D34473451345B3465346F34793464
:100C400084348E349834A334AD34B834C334CD34C2
:100C5000D834E334ED34F83404340F341A34253402
:100C600030343B34473452345D346934A0268A1121
:100C70000310540D550D8316A500A508031D462E1F
:100C80008312CF01D001D101D20108008312A02626
:100C90008A1117300310D50CD40CD30CFF3E031D62
:100CA0004A2E53088316A0008312D017D1014F0893
:100CB0008316A100831250088316A20083125108E4
:100CC0008316A3008E30A401A502A51F742E25084B
:100CD000803A8F3E031C402E0310A40CA30CA20CE0
:100CE000A10CA50F6C2E822E183025020318402E61
:100CF000A5080319822E0310A10DA20DA30DA40DAA
:100D0000A503782E20080319902EA109A209A30992
:100D1000A409A10A0319A20A0319A30A0319A40A20
:100D200024088312D200831623088312D10083166D
:100D300022088312D000831621088312CF000800F6
:100D40004F08D3005008D4005108D500080083167E
:100D5000A001A101A201A301831252085104500471
:100D60004F040319F02E8316A401A40A8312D21B88
:100D7000C02E0310CF0DD00DD10DD20D8316B52E80
:100D800003108316A00DA10DA20DA30D831252080E
:100D90005602031DD52E51085502031DD52E5008AD
:100DA0005402031DD52E4F085302031CE82E4F0892
:100DB000D3025008031C500FD4025108031C510FDA
:100DC000D5025208031C520FD602831620140310BA
:100DD0008312D20CD10CD00CCF0C8316A40BC02ED6
:100DE000831623088312D200831622088312D100AF
:100DF000831621088312D000831620088312CF00A7
:100E000008008316A7018312D71F0E2FD609D70912
:100E1000D60A0319D70A8316A701A70A8312D91F76
:100E2000192FD809D909D80A0319D90A013083160C
:100E3000A7068316A801A9018312570856040319AF
:100E4000482F8316A601A60A8312D71B2C2F031046
:100E5000D60DD70D8316232F83160310A80DA90DC9
:100E6000831257085902031D372F56085802031CD6
:100E7000412F5608D8025708031CD903D9028316FC
:100E8000281483120310D70CD60C8316A60B2C2F14
:100E9000831627080319512FA809A909A80A0319BD
:100EA000A90A29088312D700831628088312D600BE
:100EB00008005708CF005808D0008E30D101D2006A
:100EC000D30169274F08D7005008D8005108D9002E
:100ED000080052080319712F510850044F04031DD4
:100EE0007A2FCF01D001D1010800D20A0310D10C12
:100EF000D00CCF0CFE3051050319892F752FD20A63
:100F0000CF0A0319D00A0319D10A0310D10CD00C4F
:100F1000CF0CFF3051050319932F7F2FD2030310FD
:100F2000CF0DD00DD10DD01F8E2F521CD01303101A
:100F3000D20C5208D600D501D4015408CF0455086C
:100F4000D0045608D1045308031DD1170800D50159
:100F5000D601D701510850044F040319D92FD801E5
:100F6000D80AD11BB82F0310CF0DD00DD10DB02F43
:100F70000310D50DD60DD70D51085402031DC62FF1
:100F800050085302031DC62F4F085202031CD42FD2
:100F90004F08D2025008031C500FD3025108031C03
:100FA000510AD40255140310D10CD00CCF0CD80B1D
:100FB000B82F5508CF005608D0005708D1000800B8
:100FC000D000D2014F080319F92FD101D10ACF1B4C
:100FD000EC2F0310CF0DE62F0310D20D4F08500257
:100FE000031CF62F4F08D00252140310CF0CD10B64
:060FF000EC2F520808007E
:1014B6008A1190208A158A117B208A158A11862026
:1014C6008A158A119A208A15FF308312DA00DB000A
:1014D6007F30DC00BC308316B5000630B600003025
:1014E600B7007D128B10831285108A1129208A1568
:1014F6005108DE005008DD008A1113208A15DF002E
:101506008A111E208A15E0008316310883125D02B7
:10151600E100E11F902AE109E10A3C085F02C000F0
:10152600C01F972AC009C00A3E086002C100C11F39
:101536009E2AC109C10A7D1EA22A0130A32A0030B3
:101546008316AA008312061AAA2A0130AB2A003093
:1015560083162A0603193A2B8312061A3A2B061A01
:10156600B62A7D16B72A7D12831603133508831211
:10157600CF00831636088312D000831637088312ED
:10158600D1005A08D2005B08D3005C08D4008A1147
:10159600A7278A154F08A0005008A1005108A200ED
:1015A600A3012208A3002108A2002008A100A0018F
:1015B6005F08CF00D001D101D2012308D60022084E
:1015C600D5002108D4002008D3008A11A7268A1541
:1015D6005108AF005008AE004F08AD008316013029
:1015E600AA01AB0083125F0883162A028312CF007A
:1015F60083162B08031C2B038312D000D101D01BAA
:10160600D1035108D2002308D6002208D5002108AC
:10161600D4002008D3008A11A7268A155108B200E3
:101626005008B1004F08B00020088316AA008312A4
:1016360021088316AB00831222088316AC0083129E
:1016460023088316AD0007300310AD0CAC0CAB0CB1
:10165600AA0CFF3E031D272B2C088312AC00831611
:101666002B088312AB0083162A088312AA00831262
:101676006108803A7D3E03186B2B4008803A7E3E17
:1016860003186B2B4108803A7E3E03186B2B621CB5
:101696004E2B01304F2B00308316AA008312861A78
:1016A600562B0130572B003083162A06031D6B2B51
:1016B6007D1E5F2B0130602B0030AA008312061AB4
:1016C600662B0130672B003083162A0603197F2C00
:1016D60083125E088316B20083125D088316B1007A
:1016E60083126008BE005F08BC00861A7E2B831238
:1016F60003136214812B831203136210061A852BBF
:101706007D16862B7D1283120313061E0C2C5E0893
:10171600D8005D08D7008A1159278A155708A400F2
:101726005808A5005908A6009230D600D70124080B
:10173600CF002508D0002608D1008A1136268A1542
:101746005008D9004F08D8008A1101278A15560873
:10175600B8006E30CF0038088A116D208A158316BE
:10176600AA0083122408CF002508D0002608D1003D
:101776008A1136268A154F0883162A078312B9005E
:10178600123E840085300318013EFF008A110021B5
:101796008A158316AA00AB01AB00AA018312390889
:1017A600A43E840085300318013EFF008A11002103
:1017B6008A1583162A078312A00000300318013009
:1017C60083162B078312A100A201A11BA2032208E4
:1017D600A300380AF32B0310A00DA10DA20DA30D33
:1017E600FF3E031DEE2B861A002C2208A3002108BB
:1017F600A2002008A100A0010C2C05308316AA0027
:1018060003108312A00DA10DA20DA30D8316AA0B22
:10181600032C083083125F020318132C0830DF00F4
:10182600F9305F02031C192CF830DF005F08CF0087
:10183600D001D101D2012308D6002208D500210803
:10184600D4002008D3008A11A7268A155108AF00B4
:101856005008AE004F08AD0083160130AA01AB0058
:1018660083125F0883162A028312CF0083162B0881
:10187600031C2B038312D000D101D01BD1035108C6
:10188600D2002308D6002208D5002108D40020085B
:10189600D3008A11A7268A155108B2005008B10054
:1018A6004F08B00020088316AA0083122108831669
:1018B600AB00831222088316AC008312230883161A
:1018C600AD0007300310AD0CAC0CAB0CAA0CFF3E00
:1018D600031D652C2C088312AC0083162B0883127B
:1018E600AB0083162A088312AA001630CF006008C0
:1018F6008A11E0278A15BD00FD1D882C8312300849
:10190600A7003108A80032088E2C83122D08A700E4
:101916002E08A8002F08A900782A0C1C642EFB307C
:1019260010100C108F007D308E0710147D152708BF
:10193600B3022808031C280FB4022908031C290A2D
:10194600B5022A088316AE0283122B08031C2B0F3E
:10195600AD2CAF2C8316AF0283122C08031C2C0A65
:101966008316B002831235082902031DC02C3408E1
:101976002802031DC02C33082702031CE22C083062
:10198600FD06FD1DCD2C3008A7003108A800320841
:10199600A900E02C2D08A7002E08A8002F08A900F2
:1019A6005A088316AE0083125B088316AF008312B3
:1019B6005C088316B00083120615F1278A15831674
:1019C600300883122C02031DF22C83162F08831273
:1019D6002B02031DF22C83162E0883122A020318EB
:1019E6000611061EFD1E4C2E8316B50A0319B60AED
:1019F6000319B70A4C2EFD1D0F2D3308AE278A1585
:101A0600031C350FC4020C30BA278A15031D072D97
:101A16004308B7004208322D3308D8278A15FF300D
:101A2600C501C600C700C800C9014208C60243086E
:101A3600031C430FC7024408031C440FC802450891
:101A4600031C450FC9020C30CA00490DC90CC80C4D
:101A5600C70CC60CCA0B282D4708B7004608B600A7
:101A6600592EFD1D3F2D3308D8278A150C30BA276D
:101A76008A15031D3A2D542D33085A07C2005B08F8
:101A8600C30034080318340A031DC3075C08C400E6
:101A960035080318350AC4070C30BA278A15031D02
:101AA600502D4308B7004208B600E2268A15592E83
:101AB600FD1D662D3308D8278A150B30BA278A15DF
:101AC600031D612D542D3308AE278A15031C350FCF
:101AD600C4020B30BA278A15031D6D2D542DFD1D2A
:101AE6007A2DFF3083120313B6000F30342EB60161
:101AF600B701582DFD1D882D3308D8278A150F30BC
:101B0600BA278A15031D832D912D3308AE278A1512
:101B1600F8278A15BA278A15031D8D2D4308C60096
:101B26004208C50083300310C50DC60D4607FF00E9
:101B36001230292EFD1DA82D3308D8278A150A3004
:101B4600BA278A15031DA32DB12D3308AE278A1592
:101B5600FC278A15BA278A15031DAD2D4308B70041
:101B66004208B6000130B6070318B70AF030B707C7
:101B7600B71B7A2D582DFD1DC92D3308D8278A1578
:101B86000A30BA278A15031DC42DD22D3308AE2775
:101B96008A15FC278A15BA278A15031DCE2D4308F8
:101BA600B7004208B6003708803AFF0090307F023F
:101BB600031DDF2D003036020318742D582DFD1D30
:101BC600F12DFF30B6000F30B7003308D8278A153D
:101BD6000F30BA278A15031DEC2DFE2DFF30B600F7
:101BE6000F30B7003308AE278A15F8278A15BA27AB
:101BF6008A15031DFA2D4308DE27450784000318BE
:101C0600FF0A8A1100218A15C7008A1100218A1548
:101C1600C8004708B6024808031CB703B702582D88
:101C2600FD1D1E2E3308D8278A150F30BA278A15B0
:101C3600031D192E272E3308AE278A15F8278A1575
:101C4600BA278A15031D232E4308DE27450784007D
:101C56000318FF0A8A1100218A15B6008A1100218D
:101C66008A15B700582DFD19F12D1E2EFD1DFD1CE0
:101C7600432EFD10FD268A15C0278A15E2268A15F1
:101C8600FD1D592EFD14592EFD268A15C0278A15CD
:101C9600582D83123D0884000C3004020318592E77
:101CA60000308A000310040D443E8200FD1D602EA4
:101CB600FF30B6000F30B700622EB601B7015C27C1
:101CC6008A158B1CD72E8B10061E7D1DD52E203017
:101CD6007D11FD06FD1E762E8316B501B601B701F0
:101CE60083128514D72E851083163508F000360822
:101CF600F1003708F20083125A08F3005B08F4007B
:101D06005C08F50075278A157008A0007108A10007
:101D16007208A200A3012208A3002108A20020083D
:101D2600A100A0015F08F000F101F201F301E8272C
:101D36008A1514278A157208AF007108AE0070085C
:101D4600AD000130C201C3005F084202F000430843
:101D5600031C4303F100F201F11BF2037208F300C6
:101D6600E8278A1514278A157208B2007108B1008F
:101D76007008B0002008C2002108C3002208C40071
:101D86002308C50007300310C50CC40CC30CC20CD5
:101D9600FF3E031DC62E4408AC004308AB004208B4
:101DA600AA00D72EFD11F1274E08FF004D088A0024
:101DB6004C0884004B0E8300FE0E7E0E0900103088
:101DC60083120313B7070510F00185130310B60D30
:101DD600B70D031CF22E831203130517F52E83127B
:101DE6000313051310308517F00A7002031CE82E42
:101DF600051408003A083B040319BB093A1F0030D2
:101E06003A1B8030BA063A1E00303A1A8030BA06BB
:101E1600BB1D0030BB198030BA063A0DBB0DBA0D9A
:101E26000800F901FA01FB01FC0173087204710450
:101E360070040319532FF801F80AF31B282F031017
:101E4600F00DF10DF20DF30D1F2F0310F90DFA0D24
:101E5600FB0DFC0D73087702031D3B2F72087602FB
:101E6600031D3B2F71087502031D3B2F700874027A
:101E7600031C4D2F7008F4027108031C710FF50244
:101E86007208031C720FF6027308031C730FF70225
:101E960079140310F30CF20CF10CF00CF80B282F4C
:101EA6007C08F3007B08F2007A08F1007908F0005C
:101EB60008009030B7070510F00185130310B60D22
:101EC600B70D031C6A2F8312031305176D2F831298
:101ED6000313051310308517F00A7002031C602FD8
:101EE60005140800F701F801F9017208710470047D
:101EF6000319A72FF601F60AF21B862F0310F00D21
:101F0600F10DF20D7E2F0310F70DF80DF90D720885
:101F16007502031D942F71087402031D942F700817
:101F26007302031CA22F7008F3027108031C710FC1
:101F3600F4027208031C720AF50277140310F20CFD
:101F4600F10CF00CF60B862F7708F0007808F100FC
:101F56007908F20008005A02C2005B08C300340880
:101F6600031C340FC3025C08C400350808000310C4
:101F7600C40CC30CC20CFF3E0800831203133B08BB
:101F8600B600B7013A08C200F030C301C20EC30E54
:101F9600C30542080F39C304F030C2054208B6072C
:101FA6000318B70A4308B7070800C2003408C3007D
:101FB6003508C4000800C6004208C5008130031079
:101FC600C50DC60D4607FF0012342308F700220888
:101FD600F6002108F5002008F40008005A08B300AE
:101FE6005B08B4005C08B5000800031C350FC4028A
:0A1FF6000F34031C350FC4020A3437
:02400E0038CFA9
:00000001FF
